:020000007B2E55
:08000800FF00030E8312031335
:10001000C5000A0EC600040EC7008A110A12842EFB
:100020000330D407D40CD40C7F30D4050000D40B9B
:10003000162808004908CC00CB010310CC0DCB0DCD
:10004000CC0DCB0D2D30CC070318CB0A00304B075D
:100050008A004A08CB004C0882000030CC003B30BC
:1000600034280030CC005130CB070318CC0A4C08A0
:100070008A004B088200BD34AF3411342134E5349A
:10008000E634F134E33459346934F834CB34FC3495
:10009000CF3431342334FD34EF34F934EB340034CD
:1000A00000340E34073400340634153422341E3440
:1000B000053404341C340F34083401340D34163440
:1000C00063341F340C340B341D34103409340234BF
:1000D0001434173463342034133412342334113479
:1000E0000A3403341B341834633421341A34193479
:1000F0002434F808031D7D280800F930FF3E031D55
:100100007E280000F80B7D2808005508013A0319E5
:10011000A528033A0319A828013A0319AB28073A7E
:100120000319AE28013A0319B128033A0319B42878
:10013000013A0319B7280F3A0319BA28013A0319EB
:10014000BD28033A0319C0280800831206100800CE
:100150008312051308008312861108008312061209
:100160000800831286120800831206130800831207
:1001700086130800831285100800831205110800F9
:100180008312851108005508013A0319E328033A40
:100190000319E628013A0319E928073A0319EC285C
:1001A000013A0319EF28033A0319F228013A031917
:1001B000F5280F3A0319F828013A0319FB28033AE6
:1001C0000319FE280800831206140800831205177D
:1001D0000800831286150800831206160800831291
:1001E0008616080083120617080083128617080077
:1001F00083128514080083120515080083128515E3
:10020000080083120313051008008312031305145A
:100210000800053083160313D40010200800D30112
:100220000A305302031830298313511883175008DA
:10023000530784000008D4005208D500031924296C
:100240000310D40CD5031E29541C2A29530AD500A7
:10025000C3202D29530AD50085208316D30A1029DF
:100260000921052109210121092108000921052170
:100270000921012109210800013083160313CD0053
:100280000B304D0203184A294D08D50085208316EE
:10029000CD0A402901210921052109210130CD0084
:1002A0000B304D0203185A294D08D500C320831680
:1002B000CD0A502909210800052101308316CD00FF
:1002C0000B304D0203186A294D08D500C320831650
:1002D000CD0A602909210130CD000B304D020318F1
:1002E00077294D08D50085208316CD0A6D2909216F
:1002F000012109210800CF0108304F0203188A2983
:100300004D08D0004E08D1004F08073CD2000F2105
:10031000CF0A7C29362108007E08003A0319972964
:10032000013A03199A29033A03199D29A02970302B
:10033000FE00A2297230FE00A2297430FE00A2291C
:100340007630FE005C21CC010A304C020318B12942
:100350008313C23084004C0884077E088000CC0AD6
:10036000A4290030CE00C230CD007B210921CC0170
:100370000A304C020318C5298313C23084004C088C
:10038000840700308000CC0AB8290030CE00C2308B
:10039000CD007B210921CC010A304C020318EB2946
:1003A00083134118831740084C0784000008003C61
:1003B0000318E2298313C23084004C0884074630B6
:1003C0008000E9298313C23084004C08840716306A
:1003D0008000CC0ACC290030CE00C230CD007B2179
:1003E0000921CC010A304C0203180C2A83133F1850
:1003F00083173E0884004C08CD0003104D0D840780
:100400000008CE00840A8313C23084004C0884079D
:100410004E088000CC0AF2290030CE00C230CD0058
:100420007B210921CC010A304C0203182F2A8313A7
:100430003F1883173E0884004C08CD0003104D0D73
:1004400084070008CF00840A0008CE008313C2305E
:1004500084004C0884074E088000CC0A132A003020
:10046000CE00C230CD007B213C2108004008C800EE
:100470004808093C03183E2A0A30C800C80803107F
:10048000C80D831248088316C9004808CA001A20FC
:10049000C400C5014108C8004808093C8A110A1275
:1004A0000318542A0A30C800C8080310C80D831264
:1004B00048088316C900480ACA001A20C600C701A6
:1004C000F0304405C300C901C201F0304605CA003E
:1004D000CB01CA0DCB0DCA0DCB0DCA0DCB0DCA0D6C
:1004E000CB0DF0304A05C2044B08C3040F3044055D
:1004F000CC00CD01CC0DCD0DCC0DCD0DCC0DCD0D49
:10050000CC0DCD0DF0304C05C2044D08C3040F30A6
:100510004605CE004E08C2040030C3044208C9009C
:100520004308CA000800C401C201C301C31908007E
:100530000310C20DBE0DC40D3F084402031CA22AC5
:10054000C4004214C30A962ABF01C101C001C019E8
:1005500008000310C10DFE0DBF0D3E083F02031C35
:10056000B32ABF004114C00AA72AFA010A307A024E
:1005700003184A2B8312031349088316C9007A080B
:10058000CA001A20FB0025307B028A110A120318C8
:10059000E42A83137918831778087B0784000008FE
:1005A000FC0083128313203084007B08FE007E0849
:1005B000840700088316BE008313B43084007A08D1
:1005C00084073E088000ED2A6430FC008313B430B9
:1005D00084007A0884070030800064307C020318AD
:1005E000392B7C08FE000A30BE00A4224108FD0021
:1005F0007D08C0007C08BE000A30BF00932244087A
:10060000C10036228313A03084007A08FE00031054
:100610007E0D8407840A4908BE004A0880008403CE
:100620003E088000FC088A110A120319482BFD08B5
:10063000031D482B8313A03084007A08BE000310EA
:100640003E0D84070008C100840A0F30C105000870
:100650000F39C0008313A03084007A08FE00031015
:100660007E0D8407840A40088000840341088000CE
:10067000482B8313A03084007A08FE0003107E0DFF
:100680008407840A0030BE00800184033E08800095
:10069000FA0AB62A003083160313BF00A030BE004A
:1006A000FE010030C100B430C0008C21FA010A30D4
:1006B0007A020318EB2B831249088316C9000A300B
:1006C0007A07CA001A20FB0025307B028A110A1221
:1006D0000318852B83137918831778087B07840008
:1006E0000008FC0083128313203084007B08FE0086
:1006F0007E08840700088316BE008313B43084008C
:100700007A0884073E0880008E2B6430FC00831337
:10071000B43084007A0884070030800064307C02A2
:100720000318DA2B7C08FE000A30BE00A422410820
:10073000FD007D08C0007C08BE000A30BF00932287
:100740004408C10036228313A03084007A08FE00DA
:1007500003107E0D8407840A4908BE004A08800001
:1007600084033E088000FC088A110A120319E92B51
:10077000FD08031DE92B8313A03084007A08BE0016
:1007800003103E0D84070008C100840A0F30C10524
:1007900000080F39C0008313A03084007A08FE00DF
:1007A00003107E0D8407840A4008800084034108FA
:1007B0008000E92B8313A03084007A08FE00031028
:1007C0007E0D8407840A0030BE00800184033E0849
:1007D0008000FA0A572B0030BF00A030BE00013065
:1007E000FE000030C100B430C0008C21FA010A3094
:1007F0007A0203188B2C831249088316C90014301F
:100800007A07CA001A20FB0025307B028A110A12DF
:100810000318252C83137918831778087B07840025
:100820000008FC0083128313203084007B08FE0044
:100830007E08840700088316BE008313B43084004A
:100840007A0884073E0880002E2C6430FC00831355
:10085000B43084007A0884070030800064307C0261
:1008600003187A2C7C08FE000A30BE00A42241083E
:10087000FD007D08C0007C08BE000A30BF00932246
:100880004408C10036228313A03084007A08FE0099
:1008900003107E0D8407840A4908BE004A088000C0
:1008A00084033E088000FC088A110A120319892C6F
:1008B000FD08031D892C8313A03084007A08BE0034
:1008C00003103E0D84070008C100840A0F30C105E3
:1008D00000080F39C0008313A03084007A08FE009E
:1008E00003107E0D8407840A4008800084034108B9
:1008F0008000892C8313A03084007A08FE00031046
:100900007E0D8407840A0030BE00800184033E0807
:100910008000FA0AF72B0030BF00A030BE00023082
:10092000FE000030C100B430C0008C21FA010A3052
:100930007A0203182B2D831249088316C9001E3032
:100940007A07CA001A20FB0025307B028A110A129E
:100950000318C52C83137918831778087B07840044
:100960000008FC0083128313203084007B08FE0003
:100970007E08840700088316BE008313B430840009
:100980007A0884073E088000CE2C6430FC00831374
:10099000B43084007A0884070030800064307C0220
:1009A00003181A2D7C08FE000A30BE00A42241085C
:1009B000FD007D08C0007C08BE000A30BF00932205
:1009C0004408C10036228313A03084007A08FE0058
:1009D00003107E0D8407840A4908BE004A0880007F
:1009E00084033E088000FC088A110A120319292D8D
:1009F000FD08031D292D8313A03084007A08BE0052
:100A000003103E0D84070008C100840A0F30C105A1
:100A100000080F39C0008313A03084007A08FE005C
:100A200003107E0D8407840A400880008403410877
:100A30008000292D8313A03084007A08FE00031063
:100A40007E0D8407840A0030BE00800184033E08C6
:100A50008000FA0A972C0030BF00A030BE0003309F
:100A6000FE000030C100B430C0008C2108007808BE
:100A7000003A0319512D013A0319562D033A03196F
:100A80005B2D013A0319602D073A0319642D013AD1
:100A90000319682D033A03196C2D013A0319702DBF
:100AA000742D0230F9002030FA00742D1030F90056
:100AB0000230FA00742D0130F9001030FA00742D64
:100AC000F9018830FA00742D4430F900FA01742DD0
:100AD0008830F900FA01742DF9014430FA00742DC0
:100AE0002030F9000130FA00FB010A307B020318C4
:100AF0008D2D831603138313A03084007B08FC0024
:100B000003107C0D8407840A7908FD007A088000B0
:100B100084037D088000FB0A752DFB010A307B02EF
:100B200003189D2D831603138313B43084007B08B0
:100B3000840700308000FB0A8E2DFB0104307B020D
:100B400003180800003083160313BF00A030BE0056
:100B50007B08FE000030C100B430C0008C21FB0ACD
:100B60009E2D8316031385010630860007308312FD
:100B70009F0083168C160B178B17193099002030A5
:100B80009800903083129800D101D201D001CA019F
:100B9000CB01CC01CD01CE01CF0125304F0203188E
:100BA000DA2D8313533084004F08840764308000AB
:100BB000CF0ACD2D0030F9005330F800B522831252
:100BC0004E08013A0319EE2D023A0319042E073A92
:100BD00003191C2E063A03192A2E772ECF01253031
:100BE0004F020318FC2D8313533084004F088407F1
:100BF00064308000CF0AEF2D0030F9005330F80048
:100C0000B5228312CE01772ECF0125304F02031873
:100C1000142E4F0AF8008313533084004F088407C2
:100C200078088000CF0A052E0030F9005330F80014
:100C3000B5228312CE01772E5008F8003725831293
:100C40000313D00A5008073C031CD001C830F80039
:100C50007920772ECF0125304F020318382E8313C9
:100C6000533084004F08840764308000CF0A2B2E55
:100C7000CF014B084F0203184F2E4A084F07D000F0
:100C80002530500203184D2E4F0AF80083135330BD
:100C900084005008840778088000CF0A392ECF01DD
:100CA00025304F0203185D2E8313203084004F0837
:100CB000840700308000CF0A502EF9014A084D0702
:100CC000F8000318F90A7803CF0025304F02031803
:100CD000702E8313203084004F0884070130800079
:100CE0000030F9005330F800B5228312CE01C8302D
:100CF000F8007920DF2D003083120313C800013083
:100D0000C9008A110A12B12D831203131A0883161F
:100D1000D800D901580ED6000F30D605590EF0393B
:100D2000D6040F30D6050F305805D7005608003AC4
:100D30000319AA2E013A0319B22E033A0319BB2E46
:100D4000013A0319BF2E073A0319C32E013A0319BA
:100D5000C72ECA2EF0308312CC0583165708831293
:100D6000CC04CA2E0F308312CC058316570EF039EF
:100D70008312CC04CA2E83124C08CA00CA2E8312D6
:100D80004C08CB00CA2E83124C08CD00CA2E57083F
:100D90008312CE008312981CD82E80309800903099
:100DA00098001A088316D70083121A088316D700F2
:100DB0008312470E8400460E8A00450E8300FF0E04
:040DC0007F0E090099
:02400E00183F59
:00000001FF
